:100000000C943E000C9448000C9448000C9448005A
:100010000C9448000C9448000C9448000C94480040
:100020000C9448000C9448000C9448000C94480030
:100030000C9448000C9448000C9448000C94480020
:100040000C9448000C9448000C9448000C94480010
:100050000C9448000C9448000C9448000C94480000
:100060000C9448000C9448000C9448000C944800F0
:100070000C9448000C9448000C94480011241FBEB6
:10008000CFEFCDBFDFE3DEBF0E9462000C946A00B9
:100090000C9400000B9A2FE986E891E021508040F3
:1000A0009040E1F700C000000B982FE38DE093E053
:1000B000215080409040E1F700C0000008950E9468
:1000C0004A00FDCF88ED84BF10926100039A0E9420
:0800D0004A00FDCFF894FFCFB8
:00000001FF
